 sw_emextG

 Timestamp is 548ff4ce (Tue Dec 16 17:01:02 2014)

 Preferred load address is 00100000

 Start         Length     Name                   Class
 0001:00000000 000087e8H .text                   CODE
 0001:000087e8 00000220H .text$yc                CODE
 0002:00000000 00001c54H .rdata                  DATA
 0002:00001c54 000000ccH .xdata                  DATA
 0002:00001d20 00000064H .idata$2                DATA
 0002:00001d84 00000014H .idata$3                DATA
 0002:00001d98 000001f0H .idata$4                DATA
 0002:00001f88 0000033aH .idata$6                DATA
 0002:000022d0 000000daH .edata                  DATA
 0003:00000000 000001f0H .idata$5                DATA
 0003:000001f0 00000004H .CRT$XCA                DATA
 0003:000001f4 00000004H .CRT$XCAA               DATA
 0003:000001f8 00000044H .CRT$XCU                DATA
 0003:0000023c 00000004H .CRT$XCZ                DATA
 0003:00000240 00000004H .CRT$XIA                DATA
 0003:00000244 00000004H .CRT$XIZ                DATA
 0003:00000248 00000004H .CRT$XPA                DATA
 0003:0000024c 00000004H .CRT$XPZ                DATA
 0003:00000250 00000004H .CRT$XTA                DATA
 0003:00000254 00000004H .CRT$XTZ                DATA
 0003:00000258 0000005cH .data                   DATA
 0003:000002b8 00001eb0H .bss                    DATA
 0004:00000000 00000440H .pdata                  DATA
 0005:00000000 000000a0H .rsrc$01                DATA
 0005:000000a0 000003d4H .rsrc$02                DATA

  Address         Publics by Value              Rva+Base       Lib:Object

 0000:00000000       ___safe_se_handler_count   00000000     <absolute>
 0000:00000000       ___safe_se_handler_table   00000000     <absolute>
 0001:00000000       ?SetDataTab@@YAXPAUHWND__@@@Z 00101000 f   data.obj
 0001:00000104       ?InitializeData@@YAHPAUHWND__@@@Z 00101104 f   data.obj
 0001:000003b0       ?InitDataDlg@@YAHPAUHWND__@@@Z 001013b0 f   data.obj
 0001:0000041c       ?LaunchIOTA@@YAXXZ         0010141c f   data.obj
 0001:000004cc       ?LaunchSWIOMADMClient@@YAXXZ 001014cc f   data.obj
 0001:00000580       ?WndProcData@@YAHPAUHWND__@@IIJ@Z 00101580 f   data.obj
 0001:000008bc       ?SetStaticText@@YAXPAUHWND__@@@Z 001018bc f   location.obj
 0001:0000094c       ?SetLocationVal@@YAXPAUHWND__@@@Z 0010194c f   location.obj
 0001:00000b7c       ?InitializeLocation@@YAHPAUHWND__@@@Z 00101b7c f   location.obj
 0001:00000c68       ?InitLocationDlg@@YAHPAUHWND__@@@Z 00101c68 f   location.obj
 0001:00000cdc       ?WndProcLocation@@YAHPAUHWND__@@IIJ@Z 00101cdc f   location.obj
 0001:00001058       ?ReadStrValue@@YAJPAUHKEY__@@PBG1QAGK@Z 00102058 f   ruim_call_ctrl.obj
 0001:000010d0       ?WriteStrValue@@YAJPAUHKEY__@@PBG1QAGK@Z 001020d0 f   ruim_call_ctrl.obj
 0001:0000115c       ?Init_RUIM_CALL_CTRL_Dlg@@YAHPAUHWND__@@@Z 0010215c f   ruim_call_ctrl.obj
 0001:000012d8       ?SendDialStr@@YAXPAG0@Z    001022d8 f   ruim_call_ctrl.obj
 0001:000013bc       ?Update_RUIM_CALL_CTRL_Dlg@@YAHPAUHWND__@@@Z 001023bc f   ruim_call_ctrl.obj
 0001:000016f4       ?WndProc_RUIM_CALL_CTRL_Dlg@@YAHPAUHWND__@@IIJ@Z 001026f4 f   ruim_call_ctrl.obj
 0001:00001ab0       ??0ASCII@@QAA@PAG@Z        00102ab0 f   ruim_pin.obj
 0001:00001b38       ?Update_RUIM_PIN_Dlg@@YAHPAUHWND__@@@Z 00102b38 f   ruim_pin.obj
 0001:00002228       ?Init_RUIM_PIN_Dlg@@YAHPAUHWND__@@@Z 00103228 f   ruim_pin.obj
 0001:000022b0       ?HandlePIN1Action1@@YAHPAUHWND__@@@Z 001032b0 f   ruim_pin.obj
 0001:0000275c       ?HandlePIN1Action2@@YAHPAUHWND__@@@Z 0010375c f   ruim_pin.obj
 0001:00002920       ?WndProc_RUIM_PIN_Dlg@@YAHPAUHWND__@@IIJ@Z 00103920 f   ruim_pin.obj
 0001:00002b80       ?SetRoamingOption@@YAHPAK@Z 00103b80 f   Sprint_roaming_option.obj
 0001:00002c58       ?GetRoamingOption@@YAHPAK@Z 00103c58 f   Sprint_roaming_option.obj
 0001:00002d48       ?Init_SPRINT_ROAMING_OPTION_Dlg@@YAHPAUHWND__@@@Z 00103d48 f   Sprint_roaming_option.obj
 0001:00002dc0       ?Update_SPRINT_ROAMING_OPTION_Dlg@@YAHPAUHWND__@@@Z 00103dc0 f   Sprint_roaming_option.obj
 0001:00002f50       ?WndProc_SPRINT_ROAMING_OPTION_Dlg@@YAHPAUHWND__@@IIJ@Z 00103f50 f   Sprint_roaming_option.obj
 0001:00003300       ?GetResourceHandle@@YAPAUHINSTANCE__@@XZ 00104300 f   sw_emext.obj
 0001:00003310       ?GetCarrier@@YAKXZ         00104310 f   sw_emext.obj
 0001:00003320       ?InitializeGlobalVars@@YAXXZ 00104320 f   sw_emext.obj
 0001:00003390       ?SetWindowTopMost@@YAJPAUHWND__@@@Z 00104390 f   sw_emext.obj
 0001:00003404       ?AddRef@PluginFactory@@UAAKXZ 00104404 f i sw_emext.obj
 0001:00003418       ?Release@PluginFactory@@UAAKXZ 00104418 f i sw_emext.obj
 0001:0000344c       ?LockServer@PluginFactory@@UAAJH@Z 0010444c f   sw_emext.obj
 0001:00003470       DllCanUnloadNow            00104470 f   sw_emext.obj
 0001:00003494       DllRegisterServer          00104494 f   sw_emext.obj
 0001:00003610       DllUnregisterServer        00104610 f   sw_emext.obj
 0001:00003658       ??1CSW_SysSettings@@QAA@XZ 00104658 f   sw_emext.obj
 0001:000036cc       ?AddRef@CSW_SysSettings@@UAAKXZ 001046cc f i sw_emext.obj
 0001:000036e0       ?QueryInterface@CSW_SysSettings@@UAAJABU_GUID@@PAPAX@Z 001046e0 f   sw_emext.obj
 0001:00003824       ?PropPageProc@@YAHPAUHWND__@@IIJ@Z 00104824 f   sw_emext.obj
 0001:00003d78       ?PropSheetCallback@@YAIPAUHWND__@@IPAU_PROPSHEETPAGEW@@@Z 00104d78 f   sw_emext.obj
 0001:00003d88       ?AddPages@CSW_SysSettings@@UAAJP6AHPAU_PSP@@J@ZJ@Z 00104d88 f   sw_emext.obj
 0001:000042cc       ?ReplacePage@CSW_SysSettings@@UAAJIP6AHPAU_PSP@@J@ZJ@Z 001052cc f   sw_emext.obj
 0001:000042e0       ?SWDialExtERIWndProc@@YAJPAUHWND__@@IIJ@Z 001052e0 f   sw_emext.obj
 0001:00004450       ?CreateERIWindow@@YAJPAUHWND__@@PAPAU1@@Z 00105450 f   sw_emext.obj
 0001:0000454c       ?IsUserInActivecall@@YAHXZ 0010554c f   sw_emext.obj
 0001:00004580       ?GetStatus@@YAXXZ          00105580 f   sw_emext.obj
 0001:000045a8       ?SetLocationMode@@YAHK@Z   001055a8 f   sw_emext.obj
 0001:000045c8       ?SetPreferredPrivacyMode@@YAHK@Z 001055c8 f   sw_emext.obj
 0001:000045e8       ?SetRoamingMode@@YAHK@Z    001055e8 f   sw_emext.obj
 0001:00004608       ?GetRoamingMode@@YAHXZ     00105608 f   sw_emext.obj
 0001:0000464c       ?GetLocationStatus@@YAHXZ  0010564c f   sw_emext.obj
 0001:00004690       ?GetRoamStatus@@YAHXZ      00105690 f   sw_emext.obj
 0001:000046d4       ?GetPreferredPrivacyMode@@YAHXZ 001056d4 f   sw_emext.obj
 0001:00004718       ?LaunchAAM@@YAKPAX@Z       00105718 f   sw_emext.obj
 0001:000047a8       DllMain                    001057a8 f   sw_emext.obj
 0001:00004858       ?Initialize@CSW_SysSettings@@UAAJPFBU_ITEMIDLIST@@PAUIDataObject@@PAUHKEY__@@@Z 00105858 f   sw_emext.obj
 0001:00004898       ?SetSite@CSW_SysSettings@@UAAJPAUIUnknown@@@Z 00105898 f   sw_emext.obj
 0001:000048e8       ?GetSite@CSW_SysSettings@@UAAJABU_GUID@@PAPAX@Z 001058e8 f   sw_emext.obj
 0001:00004910       ?GetTypeInfoCount@CSW_SysSettings@@UAAJPAI@Z 00105910 f   sw_emext.obj
 0001:00004920       ?GetTypeInfo@CSW_SysSettings@@UAAJIKPAPAUITypeInfo@@@Z 00105920 f   sw_emext.obj
 0001:0000492c       ?GetIDsOfNames@CSW_SysSettings@@UAAJABU_GUID@@PAPAGIKPAJ@Z 0010592c f   sw_emext.obj
 0001:00004940       ?Invoke@CSW_SysSettings@@UAAJJABU_GUID@@KGPAUtagDISPPARAMS@@PAUtagVARIANT@@PAUtagEXCEPINFO@@PAI@Z 00105940 f   sw_emext.obj
 0001:00004b34       LoadOemDataIcon            00105b34 f   sw_emext.obj
 0001:00004c18       FreeOemDataIcon            00105c18 f   sw_emext.obj
 0001:00004c64       ?QueryInterface@CSW_SysSettings@@W7AAJABU_GUID@@PAPAX@Z 00105c64 f i sw_emext.obj
 0001:00004c6c       ?QueryInterface@CSW_SysSettings@@WM@AAJABU_GUID@@PAPAX@Z 00105c6c f i sw_emext.obj
 0001:00004c74       ?AddRef@CSW_SysSettings@@W3AAKXZ 00105c74 f i sw_emext.obj
 0001:00004c7c       ?AddRef@CSW_SysSettings@@W7AAKXZ 00105c7c f i sw_emext.obj
 0001:00004c84       ?AddRef@CSW_SysSettings@@WM@AAKXZ 00105c84 f i sw_emext.obj
 0001:00004c8c       ?QueryInterface@CSW_SysSettings@@W3AAJABU_GUID@@PAPAX@Z 00105c8c f i sw_emext.obj
 0001:00004c94       ?InitializeRilValues@@YAXXZ 00105c94 f   sw_emext.obj
 0001:00004cd4       ??_GPluginFactory@@UAAPAXI@Z 00105cd4 f i sw_emext.obj
 0001:00004cd4       ??_EPluginFactory@@UAAPAXI@Z 00105cd4 f i sw_emext.obj
 0001:00004cf8       ?QueryInterface@PluginFactory@@UAAJABU_GUID@@PAPAX@Z 00105cf8 f   sw_emext.obj
 0001:00004d6c       ??0CSW_SysSettings@@QAA@XZ 00105d6c f   sw_emext.obj
 0001:00004de4       ?Release@CSW_SysSettings@@UAAKXZ 00105de4 f i sw_emext.obj
 0001:00004e24       ?CreateInstance@PluginFactory@@UAAJPAUIUnknown@@ABU_GUID@@PAPAX@Z 00105e24 f   sw_emext.obj
 0001:00004ee0       DllGetClassObject          00105ee0 f   sw_emext.obj
 0001:00004f90       ?Release@CSW_SysSettings@@W3AAKXZ 00105f90 f i sw_emext.obj
 0001:00004f98       ?Release@CSW_SysSettings@@W7AAKXZ 00105f98 f i sw_emext.obj
 0001:00004fa0       ?Release@CSW_SysSettings@@WM@AAKXZ 00105fa0 f i sw_emext.obj
 0001:00004fb0       ?PopulateVZWSysTab@@YAXPAUHWND__@@@Z 00105fb0 f   syssettings.obj
 0001:0000539c       ?PopulatePCSSysTab@@YAXPAUHWND__@@@Z 0010639c f   syssettings.obj
 0001:00005688       ?PopulateGenSysTab@@YAXPAUHWND__@@@Z 00106688 f   syssettings.obj
 0001:00005a70       ?SetPreferredPrivacyMode@@YAXPAUHWND__@@@Z 00106a70 f   syssettings.obj
 0001:00005b28       ?SetRoamingVal@@YAXPAUHWND__@@@Z 00106b28 f   syssettings.obj
 0001:00005ef4       ?InitializeSysSettings@@YAHPAUHWND__@@@Z 00106ef4 f   syssettings.obj
 0001:00006068       ?InitSysSettingsDlg@@YAHPAUHWND__@@@Z 00107068 f   syssettings.obj
 0001:000060d4       ?WndProcSysSettings@@YAHPAUHWND__@@IIJ@Z 001070d4 f   syssettings.obj
 0001:00006414       ?InitializeVersionInfoDlg@@YAHPAUHWND__@@AAUtagRILVERNOINFO@@@Z 00107414 f   versioninfo.obj
 0001:00006b48       ?InitVersionInfoDlg@@YAHPAUHWND__@@@Z 00107b48 f   versioninfo.obj
 0001:00006be0       ?WndProcVersionInfoDlg@@YAHPAUHWND__@@IIJ@Z 00107be0 f   versioninfo.obj
 0001:00006d28       DestroyPropertySheetPage   00107d28 f   commctrl:commctrl.dll
 0001:00006d38       CreatePropertySheetPageW   00107d38 f   commctrl:commctrl.dll
 0001:00006d48       UpdateWindow               00107d48 f   coredll:COREDLL.dll
 0001:00006d58       EnableWindow               00107d58 f   coredll:COREDLL.dll
 0001:00006d68       GetDlgItem                 00107d68 f   coredll:COREDLL.dll
 0001:00006d78       ShowWindow                 00107d78 f   coredll:COREDLL.dll
 0001:00006d88       SetWindowTextW             00107d88 f   coredll:COREDLL.dll
 0001:00006d98       LoadStringW                00107d98 f   coredll:COREDLL.dll
 0001:00006da8       wcscat                     00107da8 f   coredll:COREDLL.dll
 0001:00006db8       MessageBoxW                00107db8 f   coredll:COREDLL.dll
 0001:00006dc8       GetLastError               00107dc8 f   coredll:COREDLL.dll
 0001:00006dd8       CreateProcessW             00107dd8 f   coredll:COREDLL.dll
 0001:00006de8       SetFocus                   00107de8 f   coredll:COREDLL.dll
 0001:00006df8       EndDialog                  00107df8 f   coredll:COREDLL.dll
 0001:00006e08       swprintf                   00107e08 f   coredll:COREDLL.dll
 0001:00006e18       RegisterClassW             00107e18 f   coredll:COREDLL.dll
 0001:00006e28       GetStockObject             00107e28 f   coredll:COREDLL.dll
 0001:00006e38       memset                     00107e38 f   coredll:COREDLL.dll
 0001:00006e48       RegisterWindowMessageW     00107e48 f   coredll:COREDLL.dll
 0001:00006e58       SetWindowPos               00107e58 f   coredll:COREDLL.dll
 0001:00006e68       GetClientRect              00107e68 f   coredll:COREDLL.dll
 0001:00006e78       SendMessageW               00107e78 f   coredll:COREDLL.dll
 0001:00006e88       SendDlgItemMessageW        00107e88 f   coredll:COREDLL.dll
 0001:00006e98       RegCloseKey                00107e98 f   coredll:COREDLL.dll
 0001:00006ea8       RegQueryValueExW           00107ea8 f   coredll:COREDLL.dll
 0001:00006eb8       RegOpenKeyExW              00107eb8 f   coredll:COREDLL.dll
 0001:00006ec8       RegSetValueExW             00107ec8 f   coredll:COREDLL.dll
 0001:00006ed8       RegCreateKeyExW            00107ed8 f   coredll:COREDLL.dll
 0001:00006ee8       NKDbgPrintfW               00107ee8 f   coredll:COREDLL.dll
 0001:00006ef8       wsprintfW                  00107ef8 f   coredll:COREDLL.dll
 0001:00006f08       _isctype                   00107f08 f   coredll:COREDLL.dll
 0001:00006f18       wcslen                     00107f18 f   coredll:COREDLL.dll
 0001:00006f28       KillTimer                  00107f28 f   coredll:COREDLL.dll
 0001:00006f38       SetTimer                   00107f38 f   coredll:COREDLL.dll
 0001:00006f48       GetWindowTextW             00107f48 f   coredll:COREDLL.dll
 0001:00006f58       malloc                     00107f58 f   coredll:COREDLL.dll
 0001:00006f68       WideCharToMultiByte        00107f68 f   coredll:COREDLL.dll
 0001:00006f78       free                       00107f78 f   coredll:COREDLL.dll
 0001:00006f88       strcpy                     00107f88 f   coredll:COREDLL.dll
 0001:00006f98       memcpy                     00107f98 f   coredll:COREDLL.dll
 0001:00006fa8       LoadLibraryW               00107fa8 f   coredll:COREDLL.dll
 0001:00006fb8       GetWindowRect              00107fb8 f   coredll:COREDLL.dll
 0001:00006fc8       SetWindowLongW             00107fc8 f   coredll:COREDLL.dll
 0001:00006fd8       GetWindowLongW             00107fd8 f   coredll:COREDLL.dll
 0001:00006fe8       memcmp                     00107fe8 f   coredll:COREDLL.dll
 0001:00006ff8       GetModuleFileNameW         00107ff8 f   coredll:COREDLL.dll
 0001:00007008       GetModuleHandleW           00108008 f   coredll:COREDLL.dll
 0001:00007018       RegDeleteKeyW              00108018 f   coredll:COREDLL.dll
 0001:00007028       _purecall                  00108028 f   coredll:COREDLL.dll
 0001:00007038       PostMessageW               00108038 f   coredll:COREDLL.dll
 0001:00007048       RemoveProp                 00108048 f   coredll:COREDLL.dll
 0001:00007058       GetActiveWindow            00108058 f   coredll:COREDLL.dll
 0001:00007068       wcscpy                     00108068 f   coredll:COREDLL.dll
 0001:00007078       EndPaint                   00108078 f   coredll:COREDLL.dll
 0001:00007088       DrawTextW                  00108088 f   coredll:COREDLL.dll
 0001:00007098       ExtTextOutW                00108098 f   coredll:COREDLL.dll
 0001:000070a8       BeginPaint                 001080a8 f   coredll:COREDLL.dll
 0001:000070b8       DefWindowProcW             001080b8 f   coredll:COREDLL.dll
 0001:000070c8       InvalidateRect             001080c8 f   coredll:COREDLL.dll
 0001:000070d8       CreateWindowExW            001080d8 f   coredll:COREDLL.dll
 0001:000070e8       CreateThread               001080e8 f   coredll:COREDLL.dll
 0001:000070f8       LoadIconW                  001080f8 f   coredll:COREDLL.dll
 0001:00007108       DestroyIcon                00108108 f   coredll:COREDLL.dll
 0001:00007118       ??3@YAXPAX@Z               00108118 f   coredll:COREDLL.dll
 0001:00007128       ??2@YAPAXI@Z               00108128 f   coredll:COREDLL.dll
 0001:00007138       wcsncpy                    00108138 f   coredll:COREDLL.dll
 0001:00007148       tapiRequestMakeCallW       00108148 f   cellcore:cellcore.dll
 0001:00007158       _DllMainCRTStartup         00108158 f   corelibc:pegdmain.obj
 0001:000071f0       __security_check_cookie    001081f0     corelibc:armsecgs.obj
 0001:00007204       __gsfailure                00108204     corelibc:armsecgs.obj
 0001:00007248       _cinit                     00108248 f   corelibc:crt0dat.obj
 0001:000073b8       _cexit                     001083b8 f   corelibc:crt0dat.obj
 0001:000073d4       __security_init_cookie     001083d4 f   corelibc:seccinit.obj
 0001:00007424       __GSHandlerCheckCommon     00108424 f   LIBCMT:gshandler.obj
 0001:0000746c       __GSHandlerCheck           0010846c f   LIBCMT:gshandler.obj
 0001:000074a4       __FrameUnwindToState       001084a4 f   LIBCMT:frame_ce.obj
 0001:0000781c       ?_DestructExceptionObject@@YAXPAUEHExceptionRecord@@E@Z 0010881c f   LIBCMT:frame_ce.obj
 0001:00007888       ?_OffsetToAddress@@YAPAXHPAKK@Z 00108888 f   LIBCMT:frame_ce.obj
 0001:000078d4       ?FindFrameInfo@@YAPAU_FrameInfo@@PAK@Z 001088d4 f   LIBCMT:frame_ce.obj
 0001:00007914       ?FindCatchFrameInfo@@YAPAU_FrameInfo@@PAK@Z 00108914 f   LIBCMT:frame_ce.obj
 0001:00007954       ?_GetRangeOfTrysToCheck@@YAPBU_s_TryBlockMapEntry@@PBU_s_FuncInfo@@HHPAI1@Z 00108954 f   LIBCMT:frame_ce.obj
 0001:00008360       __InternalCxxFrameHandler  00109360 f   LIBCMT:frame_ce.obj
 0001:000084b8       __CxxFrameHandler3         001094b8 f   LIBCMT:frame_ce.obj
 0001:000084f0       GetCRTStorage              001094f0 f   LIBCMT:corecrt.obj
 0001:000085bc       _CallSettingFrame          001095bc     LIBCMT:handlers_arm.obj
 0001:00008600       ?FindFrameForUnwind@@YAPAKPAKPBU_s_FuncInfo@@@Z 00109600 f   LIBCMT:mdframe_arm.obj
 0001:00008648       ?FindCatchFrame@@YAPAKPAKK@Z 00109648 f   LIBCMT:mdframe_arm.obj
 0001:00008694       ?AdjustFrameForCatch@@YAPAKPAKPBU_s_FuncInfo@@@Z 00109694 f   LIBCMT:mdframe_arm.obj
 0001:000086cc       ?GetCurrentState@@YAHPAKPAU_DISPATCHER_CONTEXT@@PBU_s_FuncInfo@@@Z 001096cc f   LIBCMT:ehstate_arm_mips.obj
 0001:00008728       __report_gsfailure         00109728 f   coredll:COREDLL.dll
 0001:00008738       LocalFree                  00109738 f   coredll:COREDLL.dll
 0001:00008748       __security_gen_cookie      00109748 f   coredll:COREDLL.dll
 0001:00008758       strcmp                     00109758 f   coredll:COREDLL.dll
 0001:00008768       ?terminate@std@@YAXXZ      00109768 f   coredll:COREDLL.dll
 0001:00008778       __C_specific_handler       00109778 f   coredll:COREDLL.dll
 0001:00008788       memmove                    00109788 f   coredll:COREDLL.dll
 0001:00008798       TlsCall                    00109798 f   coredll:COREDLL.dll
 0001:000087a8       TlsSetValue                001097a8 f   coredll:COREDLL.dll
 0001:000087b8       LocalAlloc                 001097b8 f   coredll:COREDLL.dll
 0001:000087c8       TlsGetValue                001097c8 f   coredll:COREDLL.dll
 0001:000087d8       InterlockedCompareExchange 001097d8 f   coredll:COREDLL.dll
 0002:00000000       ??_C@_1BE@PNHIJBIL@?$AAD?$AAa?$AAt?$AAa?$AAC?$AAl?$AAa?$AAs?$AAs?$AA?$AA@ 0010a000     data.obj
 0002:00000014       ??_C@_1BG@EGGALAJL@?$AA?4?$AA?2?$AAd?$AAa?$AAt?$AAa?$AA?4?$AAc?$AAp?$AAp?$AA?$AA@ 0010a014     data.obj
 0002:00000030       ??_C@_1IG@BPPADOJA@?$AAU?$AAn?$AAa?$AAb?$AAl?$AAe?$AA?5?$AAt?$AAo?$AA?5?$AAs?$AAt?$AAa?$AAr?$AAt?$AA?5?$AAC?$AAl?$AAi?$AAe?$AAn?$AAt?$AA?5?$AAI?$AAn?$AAi?$AAt?$AAi?$AAa?$AAt?$AAe?$AAd@ 0010a030     data.obj
 0002:000000b8       ??_C@_1BO@MDBFHABC@?$AAP?$AAh?$AAo?$AAn?$AAe?$AA?5?$AAS?$AAe?$AAt?$AAt?$AAi?$AAn?$AAg?$AAs?$AA?$AA@ 0010a0b8     data.obj
 0002:000000d8       ??_C@_1GO@EFOEHIG@?$AAU?$AAn?$AAa?$AAb?$AAl?$AAe?$AA?5?$AAt?$AAo?$AA?5?$AAs?$AAt?$AAa?$AAr?$AAt?$AA?5?$AAC?$AAl?$AAi?$AAe?$AAn?$AAt?$AA?5?$AAI?$AAn?$AAi?$AAt?$AAi?$AAa?$AAt?$AAe?$AAd@ 0010a0d8     data.obj
 0002:00000148       ??_C@_17MONHFMNG@?$AAp?$AAd?$AAp?$AA?$AA@ 0010a148     data.obj
 0002:00000150       ??_C@_1DI@GBDICIOO@?$AA?2?$AAW?$AAi?$AAn?$AAd?$AAo?$AAw?$AAs?$AA?2?$AAI?$AAO?$AAT?$AAA?$AAT?$AAh?$AAi?$AAn?$AAC?$AAl?$AAi?$AAe?$AAn?$AAt?$AA?4?$AAe?$AAx?$AAe?$AA?$AA@ 0010a150     data.obj
 0002:00000188       ??_C@_1GI@PKBHFGDE@?$AAU?$AAn?$AAa?$AAb?$AAl?$AAe?$AA?5?$AAt?$AAo?$AA?5?$AAs?$AAt?$AAa?$AAr?$AAt?$AA?5?$AAC?$AAl?$AAi?$AAe?$AAn?$AAt?$AA?5?$AAI?$AAn?$AAi?$AAt?$AAi?$AAa?$AAt?$AAe?$AAd@ 0010a188     data.obj
 0002:000001f0       ??_C@_1GA@IDJKMLOC@?$AAU?$AAn?$AAa?$AAb?$AAl?$AAe?$AA?5?$AAt?$AAo?$AA?5?$AAs?$AAt?$AAa?$AAr?$AAt?$AA?5?$AAC?$AAl?$AAi?$AAe?$AAn?$AAt?$AA?5?$AAI?$AAn?$AAi?$AAt?$AAi?$AAa?$AAt?$AAe?$AAd@ 0010a1f0     data.obj
 0002:00000250       ??_C@_1DI@FECFHFLI@?$AA?2?$AAW?$AAi?$AAn?$AAd?$AAo?$AAw?$AAs?$AA?2?$AAG?$AAo?$AAb?$AAi?$AAA?$AAc?$AAt?$AAi?$AAv?$AAa?$AAt?$AAi?$AAo?$AAn?$AA?4?$AAe?$AAx?$AAe?$AA?$AA@ 0010a250     data.obj
 0002:00000288       ??_C@_1CG@EGADBIMN@?$AAI?$AAn?$AAi?$AAt?$AAD?$AAa?$AAt?$AAa?$AAD?$AAl?$AAg?$AA?5?$AAF?$AAa?$AAi?$AAl?$AAe?$AAd?$AA?$AA@ 0010a288     data.obj
 0002:000002b0       ??_C@_11LOCGONAA@?$AA?$AA@ 0010a2b0     data.obj
 0002:000002b4       ??_C@_1CG@POBHOMMK@?$AAR?$AAI?$AAL?$AA_?$AAS?$AAT?$AAA?$AAT?$AAU?$AAS?$AA_?$AAC?$AAH?$AAA?$AAN?$AAG?$AAE?$AAD?$AA?$AA@ 0010a2b4     data.obj
 0002:000002dc       ??_C@_1CC@GILNKPAL@?$AAD?$AAa?$AAt?$AAa?$AAl?$AAi?$AAs?$AAt?$AAD?$AAl?$AAg?$AAC?$AAl?$AAa?$AAs?$AAs?$AA?$AA@ 0010a2dc     datalist.obj
 0002:00000308       ??_C@_1BM@NBCLOP@?$AAL?$AAo?$AAc?$AAa?$AAt?$AAi?$AAo?$AAn?$AAC?$AAl?$AAa?$AAs?$AAs?$AA?$AA@ 0010a308     location.obj
 0002:00000324       ??_C@_1BO@LOBFKOCC@?$AA?4?$AA?2?$AAl?$AAo?$AAc?$AAa?$AAt?$AAi?$AAo?$AAn?$AA?4?$AAc?$AAp?$AAp?$AA?$AA@ 0010a324     location.obj
 0002:00000344       ??_C@_1CO@NAADAPJD@?$AAI?$AAn?$AAi?$AAt?$AAL?$AAo?$AAc?$AAa?$AAt?$AAi?$AAo?$AAn?$AAD?$AAl?$AAg?$AA?5?$AAF?$AAa?$AAi?$AAl?$AAe?$AAd?$AA?$AA@ 0010a344     location.obj
 0002:00000374       ??_C@_1CA@BLLJOMJF@?$AAP?$AAH?$AAS?$AAL?$AAi?$AAs?$AAt?$AAD?$AAl?$AAg?$AAC?$AAl?$AAa?$AAs?$AAs?$AA?$AA@ 0010a374     phs_list.obj
 0002:000003a4       ??_C@_1DA@IFALCCCH@?$AAR?$AAU?$AAI?$AAM?$AA_?$AAC?$AAA?$AAL?$AAL?$AA_?$AAC?$AAT?$AAR?$AAL?$AA_?$AAD?$AAl?$AAg?$AAC?$AAl?$AAa?$AAs?$AAs?$AA?$AA@ 0010a3a4     ruim_call_ctrl.obj
 0002:000003d4       ??_C@_1DE@EMJBEPGN@?$AA?2?$AAS?$AAt?$AAr?$AAi?$AAn?$AAg?$AAF?$AAi?$AAl?$AAe?$AAI?$AAn?$AAf?$AAo?$AA?2?$AA0?$AA4?$AA0?$AA9?$AA0?$AA4?$AAB?$AA0?$AA?2?$AA?$AA@ 0010a3d4     ruim_call_ctrl.obj
 0002:00000408       ??_C@_1CI@MHCGMGFN@?$AAF?$AAo?$AAr?$AAw?$AAa?$AAr?$AAd?$AAA?$AAl?$AAl?$AAV?$AAo?$AAi?$AAc?$AAe?$AAC?$AAa?$AAl?$AAl?$AA?$AA@ 0010a408     ruim_call_ctrl.obj
 0002:00000430       ??_C@_1BM@HJJDODHJ@?$AAF?$AAo?$AAr?$AAw?$AAa?$AAr?$AAd?$AAO?$AAn?$AAB?$AAu?$AAs?$AAy?$AA?$AA@ 0010a430     ruim_call_ctrl.obj
 0002:0000044c       ??_C@_1CE@PANGPJFM@?$AAF?$AAo?$AAr?$AAw?$AAa?$AAr?$AAd?$AAO?$AAn?$AAN?$AAo?$AAA?$AAn?$AAs?$AAw?$AAe?$AAr?$AA?$AA@ 0010a44c     ruim_call_ctrl.obj
 0002:00000470       ??_C@_1CI@DPOHACAB@?$AAF?$AAo?$AAr?$AAw?$AAa?$AAr?$AAd?$AAO?$AAn?$AAO?$AAu?$AAt?$AAO?$AAf?$AAR?$AAe?$AAa?$AAc?$AAh?$AA?$AA@ 0010a470     ruim_call_ctrl.obj
 0002:00000498       ??_C@_1GE@BNNLGEIG@?$AA?2?$AAS?$AAo?$AAf?$AAt?$AAw?$AAa?$AAr?$AAe?$AA?2?$AAS?$AAi?$AAe?$AAr?$AAr?$AAa?$AA?5?$AAW?$AAi?$AAr?$AAe?$AAl?$AAe?$AAs?$AAs?$AA?5?$AAI?$AAn?$AAc?$AA?2?$AAR?$AAI@ 0010a498     ruim_call_ctrl.obj
 0002:000004fc       ??_C@_1CE@ODCGNLLP@?$AAR?$AAU?$AAI?$AAM?$AA?5?$AAC?$AAa?$AAl?$AAl?$AA?5?$AAC?$AAo?$AAn?$AAt?$AAr?$AAo?$AAl?$AA?$AA@ 0010a4fc     ruim_call_ctrl.obj
 0002:00000520       ??_C@_1CO@LLMCFIKC@?$AAI?$AAn?$AAc?$AAo?$AAr?$AAr?$AAe?$AAc?$AAt?$AA?5?$AAp?$AAh?$AAo?$AAn?$AAe?$AA?5?$AAn?$AAu?$AAm?$AAb?$AAe?$AAr?$AA?$AA@ 0010a520     ruim_call_ctrl.obj
 0002:00000550       ??_C@_19LJDFFCJJ@?$AA?$CF?$AAs?$AA?$CF?$AAs?$AA?$AA@ 0010a550     ruim_call_ctrl.obj
 0002:00000560       ??_C@_1FI@FMBNBHOF@?$AAS?$AAe?$AAn?$AAd?$AAD?$AAi?$AAa?$AAl?$AAS?$AAt?$AAr?$AA?5?$AAs?$AAe?$AAn?$AAd?$AAi?$AAn?$AAg?$AA?5?$AAc?$AAo?$AAm?$AAm?$AAa?$AAn?$AAd?$AA?5?$AA?$CF?$AAs?$AA?0?$AA?5@ 0010a560     ruim_call_ctrl.obj
 0002:000005b8       ??_C@_1CK@HPBOBAPA@?$AA?4?$AA?2?$AAr?$AAu?$AAi?$AAm?$AA_?$AAc?$AAa?$AAl?$AAl?$AA_?$AAc?$AAt?$AAr?$AAl?$AA?4?$AAc?$AAp?$AAp?$AA?$AA@ 0010a5b8     ruim_call_ctrl.obj
 0002:000005e8       ??_C@_1EO@MCMHDFBM@?$AAc?$AAr?$AAe?$AAa?$AAt?$AAe?$AA?5?$AAg?$AA_?$AAC?$AAa?$AAl?$AAl?$AAC?$AAr?$AAl?$AAT?$AAi?$AAm?$AAe?$AAr?$AA?5?$AAt?$AAi?$AAm?$AAe?$AAr?$AA?5?$AAf?$AAa?$AAi?$AAl@ 0010a5e8     ruim_call_ctrl.obj
 0002:00000638       ??_C@_1DO@KPNAIOLL@?$AAI?$AAn?$AAi?$AAt?$AA_?$AAR?$AAU?$AAI?$AAM?$AA_?$AAC?$AAA?$AAL?$AAL?$AA_?$AAC?$AAT?$AAR?$AAL?$AA_?$AAD?$AAl?$AAg?$AA?5?$AAF?$AAa?$AAi?$AAl?$AAe?$AAd?$AA?$AA@ 0010a638     ruim_call_ctrl.obj
 0002:00000678       ??_C@_17BFNHGKPG@?$AA?$CK?$AA6?$AA8?$AA?$AA@ 0010a678     ruim_call_ctrl.obj
 0002:00000680       ??_C@_17JIKDOFC@?$AA?$CK?$AA7?$AA3?$AA?$AA@ 0010a680     ruim_call_ctrl.obj
 0002:00000688       ??_C@_13KBPCEPBF@?$AA4?$AA?$AA@ 0010a688     ruim_call_ctrl.obj
 0002:0000068c       ??_C@_15IFPGLIBE@?$AA?$CK?$AA7?$AA?$AA@ 0010a68c     ruim_call_ctrl.obj
 0002:00000694       ??_C@_17JEFNAGOL@?$AA?$CK?$AA7?$AA4?$AA?$AA@ 0010a694     ruim_call_ctrl.obj
 0002:0000069c       ??_C@_17LBDGFJDH@?$AA?$CK?$AA7?$AA2?$AA?$AA@ 0010a69c     ruim_call_ctrl.obj
 0002:000006a4       ??_C@_13COJANIEC@?$AA0?$AA?$AA@ 0010a6a4     ruim_call_ctrl.obj
 0002:000006a8       ??_C@_17CBDFPAMM@?$AA?$CK?$AA9?$AA0?$AA?$AA@ 0010a6a8     ruim_call_ctrl.obj
 0002:000006b0       ??_C@_17ILDMDIEH@?$AA?$CK?$AA9?$AA2?$AA?$AA@ 0010a6b0     ruim_call_ctrl.obj
 0002:000006b8       ??_C@_1BO@NKICKCPO@?$AAR?$AAI?$AAL?$AA_?$AAD?$AAB?$AAG?$AA_?$AAN?$AAO?$AAT?$AAI?$AAF?$AAY?$AA?$AA@ 0010a6b8     ruim_call_ctrl.obj
 0002:000006d8       ??_C@_1CA@BMOKIJOD@?$AAR?$AAI?$AAL?$AA_?$AAS?$AAE?$AAT?$AA_?$AAE?$AAR?$AAI?$AAT?$AAE?$AAX?$AAT?$AA?$AA@ 0010a6d8     ruim_call_ctrl.obj
 0002:000006f8       ??_C@_1CI@GFFCIEDP@?$AAP?$AAe?$AAr?$AAm?$AAa?$AAn?$AAe?$AAn?$AAt?$AAl?$AAy?$AA?5?$AAb?$AAl?$AAo?$AAc?$AAk?$AAe?$AAd?$AA?$AA@ 0010a6f8     ruim_pin.obj
 0002:00000720       ??_C@_1BA@BNFIHHGN@?$AAB?$AAl?$AAo?$AAc?$AAk?$AAe?$AAd?$AA?$AA@ 0010a720     ruim_pin.obj
 0002:00000730       ??_C@_1BC@FGCJDNHA@?$AAD?$AAi?$AAs?$AAa?$AAb?$AAl?$AAe?$AAd?$AA?$AA@ 0010a730     ruim_pin.obj
 0002:00000744       ??_C@_1BC@HEOALF@?$AAV?$AAe?$AAr?$AAi?$AAf?$AAi?$AAe?$AAd?$AA?$AA@ 0010a744     ruim_pin.obj
 0002:00000758       ??_C@_1BG@GAKIPDFC@?$AAP?$AAi?$AAn?$AA?5?$AAL?$AAo?$AAc?$AAk?$AAe?$AAd?$AA?$AA@ 0010a758     ruim_pin.obj
 0002:00000770       ??_C@_1BA@LEPJIIOK@?$AAU?$AAn?$AAk?$AAn?$AAo?$AAw?$AAn?$AA?$AA@ 0010a770     ruim_pin.obj
 0002:00000780       ??_C@_1CE@FHMPNJBL@?$AAR?$AAU?$AAI?$AAM?$AA_?$AAP?$AAI?$AAN?$AA_?$AAD?$AAl?$AAg?$AAC?$AAl?$AAa?$AAs?$AAs?$AA?$AA@ 0010a780     ruim_pin.obj
 0002:000007a4       ??_C@_1CO@IEAPNEPJ@?$AAI?$AAn?$AAv?$AAa?$AAl?$AAi?$AAd?$AA?5?$AAS?$AAI?$AAM?$AA?5?$AAo?$AAr?$AA?5?$AAN?$AAo?$AA?5?$AAS?$AAI?$AAM?$AA?4?$AA?$AA@ 0010a7a4     ruim_pin.obj
 0002:000007d4       ??_C@_1CC@HFAKDMDE@?$AAS?$AAI?$AAM?$AA?5?$AAc?$AAa?$AAr?$AAd?$AA?5?$AAu?$AAn?$AAk?$AAn?$AAo?$AAw?$AAn?$AA?$AA@ 0010a7d4     ruim_pin.obj
 0002:000007f8       ??_C@_1FI@CIGELBEB@?$AAP?$AAl?$AAe?$AAa?$AAs?$AAe?$AA?5?$AAi?$AAn?$AAp?$AAu?$AAt?$AA?5?$AAy?$AAo?$AAu?$AAr?$AA?5?$AAP?$AAI?$AAN?$AA?5?$AAc?$AAo?$AAd?$AAe?$AA?4?$AA?5?$AAR?$AAe?$AAt?$AAr@ 0010a7f8     ruim_pin.obj
 0002:00000850       ??_C@_1O@LEPOPAGP@?$AAV?$AAe?$AAr?$AAi?$AAf?$AAy?$AA?$AA@ 0010a850     ruim_pin.obj
 0002:00000860       ??_C@_1HI@CNMPCCM@?$AAY?$AAo?$AAu?$AA?5?$AAc?$AAa?$AAn?$AA?5?$AAd?$AAi?$AAs?$AAa?$AAb?$AAl?$AAe?$AA?5?$AAS?$AAI?$AAM?$AA?5?$AAl?$AAo?$AAc?$AAk?$AA?5?$AAw?$AAi?$AAt?$AAh?$AA?5?$AAt?$AAh@ 0010a860     ruim_pin.obj
 0002:000008d8       ??_C@_1BA@EHHBCNCC@?$AAD?$AAi?$AAs?$AAa?$AAb?$AAl?$AAe?$AA?$AA@ 0010a8d8     ruim_pin.obj
 0002:000008e8       ??_C@_1HG@GAHIPNKC@?$AAY?$AAo?$AAu?$AA?5?$AAc?$AAa?$AAn?$AA?5?$AAe?$AAn?$AAa?$AAb?$AAl?$AAe?$AA?5?$AAS?$AAI?$AAM?$AA?5?$AAl?$AAo?$AAc?$AAk?$AA?5?$AAw?$AAi?$AAt?$AAh?$AA?5?$AAt?$AAh?$AAe@ 0010a8e8     ruim_pin.obj
 0002:00000960       ??_C@_1O@PFBIKACK@?$AAE?$AAn?$AAa?$AAb?$AAl?$AAe?$AA?$AA@ 0010a960     ruim_pin.obj
 0002:00000970       ??_C@_17JMGHKHPK@?$AAP?$AAI?$AAN?$AA?$AA@ 0010a970     ruim_pin.obj
 0002:00000978       ??_C@_1IA@KOOILHFJ@?$AAY?$AAo?$AAu?$AA?5?$AAc?$AAa?$AAn?$AA?5?$AAu?$AAn?$AAb?$AAl?$AAo?$AAc?$AAk?$AA?5?$AAt?$AAh?$AAe?$AA?5?$AAS?$AAI?$AAM?$AA?5?$AAc?$AAa?$AAr?$AAd?$AA?5?$AAw?$AAi?$AAt@ 0010a978     ruim_pin.obj
 0002:000009f8       ??_C@_1BA@ICDMNCPJ@?$AAU?$AAn?$AAb?$AAl?$AAo?$AAc?$AAk?$AA?$AA@ 0010a9f8     ruim_pin.obj
 0002:00000a08       ??_C@_17NPKNJFCI@?$AAP?$AAU?$AAK?$AA?$AA@ 0010aa08     ruim_pin.obj
 0002:00000a10       ??_C@_1BA@MPDLJHI@?$AAN?$AAe?$AAw?$AA?5?$AAP?$AAI?$AAN?$AA?$AA@ 0010aa10     ruim_pin.obj
 0002:00000a20       ??_C@_1LM@BKLMLGBK@?$AAY?$AAo?$AAu?$AAr?$AA?5?$AAS?$AAI?$AAM?$AA?5?$AAc?$AAa?$AAr?$AAd?$AA?5?$AAi?$AAs?$AA?5?$AAp?$AAe?$AAr?$AAm?$AAa?$AAn?$AAe?$AAn?$AAt?$AAl?$AAy?$AA?5?$AAb?$AAl?$AAo@ 0010aa20     ruim_pin.obj
 0002:00000ae0       ??_C@_1HA@HGKAHJMN@?$AAc?$AAu?$AAr?$AAR?$AAT?$AAR?$AAE?$AA?3?$AA?$CF?$AAd?$AA?0?$AA?5?$AAs?$AAl?$AAo?$AAt?$AA?3?$AA?$CF?$AAd?$AA?5?$AAa?$AAp?$AAp?$AAl?$AA?3?$AA?$CF?$AAd?$AA?0?$AA?5?$AAu?$AAn?$AAi@ 0010aae0     ruim_pin.obj
 0002:00000b50       ??_C@_1DG@HFHNGJDA@?$AAP?$AAh?$AAo?$AAn?$AAe?$AA?5?$AAi?$AAs?$AA?5?$AAn?$AAo?$AAt?$AA?5?$AAi?$AAn?$AA?5?$AAR?$AAU?$AAI?$AAM?$AA?5?$AAm?$AAo?$AAd?$AAe?$AA?4?$AA?$AA@ 0010ab50     ruim_pin.obj
 0002:00000b88       ??_C@_1BO@CNMHOIBI@?$AA?4?$AA?2?$AAr?$AAu?$AAi?$AAm?$AA_?$AAp?$AAi?$AAn?$AA?4?$AAc?$AAp?$AAp?$AA?$AA@ 0010ab88     ruim_pin.obj
 0002:00000ba8       ??_C@_1BG@CKCODMCF@?$AAc?$AAu?$AAr?$AAR?$AAT?$AAR?$AAE?$AA?3?$AA?$CF?$AAd?$AA?$AA@ 0010aba8     ruim_pin.obj
 0002:00000bc0       ??_C@_1DC@LFENLPAM@?$AAP?$AAh?$AAo?$AAn?$AAe?$AA?5?$AAi?$AAs?$AA?5?$AAn?$AAo?$AAt?$AA?5?$AAp?$AAo?$AAw?$AAe?$AAr?$AAe?$AAd?$AA?5?$AAo?$AAn?$AA?4?$AA?$AA@ 0010abc0     ruim_pin.obj
 0002:00000bf4       ??_C@_1BA@IHNFGJPH@?$AAD?$AAi?$AAs?$AAm?$AAi?$AAs?$AAs?$AA?$AA@ 0010abf4     ruim_pin.obj
 0002:00000c04       ??_C@_1CO@BNOAEAJH@?$AAP?$AAI?$AAN?$AA?5?$AAv?$AAe?$AAr?$AAi?$AAf?$AAi?$AAe?$AAd?$AA?5?$AAc?$AAo?$AAr?$AAr?$AAe?$AAc?$AAl?$AAy?$AA?4?$AA?$AA@ 0010ac04     ruim_pin.obj
 0002:00000c34       ??_C@_1BM@DFPCOPLE@?$AAI?$AAn?$AAc?$AAo?$AAr?$AAr?$AAe?$AAc?$AAt?$AA?5?$AAP?$AAI?$AAN?$AA?$AA@ 0010ac34     ruim_pin.obj
 0002:00000c50       ??_C@_1DO@BDHAAMBN@?$AAP?$AAI?$AAN?$AA?5?$AAl?$AAo?$AAc?$AAk?$AA?5?$AAd?$AAi?$AAs?$AAa?$AAb?$AAl?$AAe?$AAd?$AA?5?$AAs?$AAu?$AAc?$AAc?$AAe?$AAs?$AAs?$AAf?$AAu?$AAl?$AAl?$AAy?$AA?$AA@ 0010ac50     ruim_pin.obj
 0002:00000c90       ??_C@_1DM@DNLGOHKB@?$AAP?$AAI?$AAN?$AA?5?$AAl?$AAo?$AAc?$AAk?$AA?5?$AAe?$AAn?$AAa?$AAb?$AAl?$AAe?$AAd?$AA?5?$AAs?$AAu?$AAc?$AAc?$AAe?$AAs?$AAs?$AAf?$AAu?$AAl?$AAl?$AAy?$AA?$AA@ 0010ac90     ruim_pin.obj
 0002:00000cd0       ??_C@_1GE@JAMBBJIM@?$AAI?$AAn?$AAc?$AAo?$AAr?$AAr?$AAe?$AAc?$AAt?$AA?5?$AAP?$AAI?$AAN?$AA?0?$AA?5?$AAe?$AAr?$AAr?$AAo?$AAr?$AA?5?$AAc?$AAo?$AAd?$AAe?$AA?3?$AA?5?$AA?$CF?$AAd?$AA?0?$AA?5?$AAr@ 0010acd0     ruim_pin.obj
 0002:00000d34       ??_C@_1DG@LNNCBHNG@?$AAP?$AAI?$AAN?$AA?5?$AAu?$AAn?$AAb?$AAl?$AAo?$AAc?$AAk?$AAe?$AAd?$AA?5?$AAs?$AAu?$AAc?$AAc?$AAe?$AAs?$AAs?$AAf?$AAu?$AAl?$AAl?$AAy?$AA?$AA@ 0010ad34     ruim_pin.obj
 0002:00000d70       ??_C@_1FM@GEBKPJNN@?$AAI?$AAn?$AAc?$AAo?$AAr?$AAr?$AAe?$AAc?$AAt?$AA?5?$AAP?$AAU?$AAK?$AA?4?$AA?5?$AAE?$AAr?$AAr?$AAo?$AAr?$AA?5?$AAc?$AAo?$AAd?$AAe?$AA?5?$AA?3?$AA?$CF?$AAd?$AA?5?$AAR?$AAe@ 0010ad70     ruim_pin.obj
 0002:00000dcc       ??_C@_1BO@GELLEJIG@?$AAP?$AAh?$AAo?$AAn?$AAe?$AA?5?$AAS?$AAe?$AAc?$AAu?$AAr?$AAi?$AAt?$AAy?$AA?$AA@ 0010adcc     ruim_pin.obj
 0002:00000dec       ??_C@_1DC@KLHGJJOM@?$AAP?$AAI?$AAN?$AA?5?$AAc?$AAh?$AAa?$AAn?$AAg?$AAe?$AAd?$AA?5?$AAs?$AAu?$AAc?$AAc?$AAe?$AAs?$AAs?$AAf?$AAu?$AAl?$AAl?$AAy?$AA?$AA@ 0010adec     ruim_pin.obj
 0002:00000e20       ??_C@_1GC@HAKPKAOE@?$AAI?$AAn?$AAc?$AAo?$AAr?$AAr?$AAe?$AAc?$AAt?$AA?5?$AAP?$AAI?$AAN?$AA?4?$AA?5?$AAE?$AAr?$AAr?$AAo?$AAr?$AA?5?$AAc?$AAo?$AAd?$AAe?$AA?5?$AA?$CF?$AA1?$AA?5?$AAR?$AAe?$AAt@ 0010ae20     ruim_pin.obj
 0002:00000e84       ??_C@_1DC@DPMIOGGC@?$AAI?$AAn?$AAi?$AAt?$AA_?$AAR?$AAU?$AAI?$AAM?$AA_?$AAP?$AAI?$AAN?$AA_?$AAD?$AAl?$AAg?$AA?5?$AAF?$AAa?$AAi?$AAl?$AAe?$AAd?$AA?$AA@ 0010ae84     ruim_pin.obj
 0002:00000eb8       ??_C@_1DO@ILONOHL@?$AAS?$AAP?$AAR?$AAI?$AAN?$AAT?$AA_?$AAR?$AAO?$AAA?$AAM?$AAI?$AAN?$AAG?$AA_?$AAO?$AAP?$AAT?$AAI?$AAO?$AAN?$AA_?$AAD?$AAl?$AAg?$AAC?$AAl?$AAa?$AAs?$AAs?$AA?$AA@ 0010aeb8     Sprint_roaming_option.obj
 0002:00000ef8       ??_C@_1CK@LDOMAMIN@?$AAG?$AAo?$AAb?$AAi?$AA?5?$AAn?$AAo?$AAt?$AA?5?$AAc?$AAo?$AAn?$AAn?$AAe?$AAc?$AAt?$AAe?$AAd?$AA?$CB?$AA?$CB?$AA?$AA@ 0010aef8     Sprint_roaming_option.obj
 0002:00000f24       ??_C@_1DI@FEKNALDL@?$AA?4?$AA?2?$AAS?$AAp?$AAr?$AAi?$AAn?$AAt?$AA_?$AAr?$AAo?$AAa?$AAm?$AAi?$AAn?$AAg?$AA_?$AAo?$AAp?$AAt?$AAi?$AAo?$AAn?$AA?4?$AAc?$AAp?$AAp?$AA?$AA@ 0010af24     Sprint_roaming_option.obj
 0002:00000f60       ??_C@_1FG@FINKMNAD@?$AAS?$AAe?$AAt?$AAC?$AAD?$AAM?$AAA?$AAN?$AAe?$AAt?$AAw?$AAo?$AAr?$AAk?$AAP?$AAa?$AAr?$AAa?$AAm?$AAe?$AAt?$AAe?$AAr?$AAs?$AA?5?$AAf?$AAa?$AAi?$AAl?$AAe?$AAd?$AA?0@ 0010af60     Sprint_roaming_option.obj
 0002:00000fb8       ??_C@_1FG@ECJGADME@?$AAG?$AAe?$AAt?$AAC?$AAD?$AAM?$AAA?$AAN?$AAe?$AAt?$AAw?$AAo?$AAr?$AAk?$AAP?$AAa?$AAr?$AAa?$AAm?$AAe?$AAt?$AAe?$AAr?$AAs?$AA?5?$AAf?$AAa?$AAi?$AAl?$AAe?$AAd?$AA?0@ 0010afb8     Sprint_roaming_option.obj
 0002:00001010       ??_C@_1BE@OIBEOKIJ@?$AAR?$AAo?$AAa?$AAm?$AAG?$AAu?$AAa?$AAr?$AAd?$AA?$AA@ 0010b010     Sprint_roaming_option.obj
 0002:00001028       ??_C@_1EK@CPPGCLPN@?$AA?2?$AAS?$AAo?$AAf?$AAt?$AAw?$AAa?$AAr?$AAe?$AA?2?$AAS?$AAi?$AAe?$AAr?$AAr?$AAa?$AA?5?$AAW?$AAi?$AAr?$AAe?$AAl?$AAe?$AAs?$AAs?$AA?5?$AAI?$AAn?$AAc?$AA?2?$AAS?$AAy@ 0010b028     Sprint_roaming_option.obj
 0002:00001078       ??_C@_1EM@DHBOCMOK@?$AAI?$AAn?$AAi?$AAt?$AA_?$AAS?$AAP?$AAR?$AAI?$AAN?$AAT?$AA_?$AAR?$AAO?$AAA?$AAM?$AAI?$AAN?$AAG?$AA_?$AAO?$AAP?$AAT?$AAI?$AAO?$AAN?$AA_?$AAD?$AAl?$AAg?$AA?5?$AAF@ 0010b078     Sprint_roaming_option.obj
 0002:000010c4       CLSID_SWEMEXTCPL           0010b0c4     sw_emext.obj
 0002:000010d4       IID_ITPCSettingsFullCustomCPL 0010b0d4     sw_emext.obj
 0002:000010e4       IID_IObjectWithSite        0010b0e4     sw_emext.obj
 0002:000010f4       GUID_NULL                  0010b0f4     sw_emext.obj
 0002:00001104       IID_IUnknown               0010b104     sw_emext.obj
 0002:00001114       IID_IClassFactory          0010b114     sw_emext.obj
 0002:00001124       IID_IMalloc                0010b124     sw_emext.obj
 0002:00001134       IID_IMarshal               0010b134     sw_emext.obj
 0002:00001144       IID_IRpcChannel            0010b144     sw_emext.obj
 0002:00001154       IID_IRpcStub               0010b154     sw_emext.obj
 0002:00001164       IID_IStubManager           0010b164     sw_emext.obj
 0002:00001174       IID_IRpcProxy              0010b174     sw_emext.obj
 0002:00001184       IID_IProxyManager          0010b184     sw_emext.obj
 0002:00001194       IID_IPSFactory             0010b194     sw_emext.obj
 0002:000011a4       IID_ILockBytes             0010b1a4     sw_emext.obj
 0002:000011b4       IID_IStorage               0010b1b4     sw_emext.obj
 0002:000011c4       IID_IStream                0010b1c4     sw_emext.obj
 0002:000011d4       IID_IEnumSTATSTG           0010b1d4     sw_emext.obj
 0002:000011e4       IID_IBindCtx               0010b1e4     sw_emext.obj
 0002:000011f4       IID_IMoniker               0010b1f4     sw_emext.obj
 0002:00001204       IID_IRunningObjectTable    0010b204     sw_emext.obj
 0002:00001214       IID_IInternalMoniker       0010b214     sw_emext.obj
 0002:00001224       IID_IRootStorage           0010b224     sw_emext.obj
 0002:00001234       IID_IDfReserved1           0010b234     sw_emext.obj
 0002:00001244       IID_IDfReserved2           0010b244     sw_emext.obj
 0002:00001254       IID_IDfReserved3           0010b254     sw_emext.obj
 0002:00001264       IID_IMessageFilter         0010b264     sw_emext.obj
 0002:00001274       CLSID_StdMarshal           0010b274     sw_emext.obj
 0002:00001284       IID_IStdMarshalInfo        0010b284     sw_emext.obj
 0002:00001294       IID_IExternalConnection    0010b294     sw_emext.obj
 0002:000012a4       ??_C@_1CA@MNHLNOBN@?$AAs?$AAw?$AAi?$AA_?$AAr?$AAi?$AAl?$AAr?$AAe?$AAs?$AAG?$AA?4?$AAd?$AAl?$AAl?$AA?$AA@ 0010b2a4     sw_emext.obj
 0002:000012c4       ??_7PluginFactory@@6B@     0010b2c4     sw_emext.obj
 0002:000012dc       ??_C@_1BM@DNHAIOIA@?$AAs?$AAw?$AA_?$AAe?$AAm?$AAe?$AAx?$AAt?$AAG?$AA?4?$AAd?$AAl?$AAl?$AA?$AA@ 0010b2dc     sw_emext.obj
 0002:000012f8       ??_C@_1BO@MNKPAJEP@?$AAI?$AAn?$AAp?$AAr?$AAo?$AAc?$AAS?$AAe?$AAr?$AAv?$AAe?$AAr?$AA3?$AA2?$AA?$AA@ 0010b2f8     sw_emext.obj
 0002:00001318       ??_C@_1BG@HFOCDLHN@?$AAS?$AAW?$AAE?$AAM?$AAE?$AAX?$AAT?$AAC?$AAP?$AAL?$AA?$AA@ 0010b318     sw_emext.obj
 0002:00001330       ??_C@_1FK@CKMIPDMF@?$AAC?$AAL?$AAS?$AAI?$AAD?$AA?2?$AA?$HL?$AA9?$AA1?$AA1?$AA3?$AAE?$AAF?$AA8?$AAF?$AA?9?$AAE?$AA0?$AAE?$AA5?$AA?9?$AA4?$AA8?$AA7?$AAB?$AA?9?$AA8?$AA5?$AA5?$AA9?$AA?9?$AAE@ 0010b330     sw_emext.obj
 0002:00001390       ??_C@_1HI@FLPJGIBE@?$AAC?$AAL?$AAS?$AAI?$AAD?$AA?2?$AA?$HL?$AA9?$AA1?$AA1?$AA3?$AAE?$AAF?$AA8?$AAF?$AA?9?$AAE?$AA0?$AAE?$AA5?$AA?9?$AA4?$AA8?$AA7?$AAB?$AA?9?$AA8?$AA5?$AA5?$AA9?$AA?9?$AAE@ 0010b390     sw_emext.obj
 0002:00001408       ??_7IShellExtInit@@6B@     0010b408     sw_emext.obj
 0002:00001418       ??_7IShellPropSheetExt@@6B@ 0010b418     sw_emext.obj
 0002:0000142c       ??_7CSW_SysSettings@@6BIObjectWithSite@@@ 0010b42c     sw_emext.obj
 0002:00001440       ??_7CSW_SysSettings@@6BIShellExtInit@@@ 0010b440     sw_emext.obj
 0002:00001450       ??_7CSW_SysSettings@@6BIDispatch@@@ 0010b450     sw_emext.obj
 0002:0000146c       ??_7CSW_SysSettings@@6BIShellPropSheetExt@@@ 0010b46c     sw_emext.obj
 0002:00001480       ??_C@_15HCBMMKJC@?$AAI?$AAD?$AA?$AA@ 0010b480     sw_emext.obj
 0002:00001488       ??_C@_1EG@NLHEHNFK@?$AAR?$AAe?$AAg?$AAi?$AAs?$AAt?$AAr?$AAy?$AA?5?$AAi?$AAs?$AA?5?$AAs?$AAe?$AAt?$AA?5?$AAt?$AAo?$AA?5?$AAh?$AAi?$AAd?$AAe?$AA?5?$AAS?$AAy?$AAs?$AAt?$AAe?$AAm?$AA?5?$AAT@ 0010b488     sw_emext.obj
 0002:000014d0       ??_C@_1EC@MIIHMILP@?$AAR?$AAe?$AAg?$AAi?$AAs?$AAt?$AAr?$AAy?$AA?5?$AAi?$AAs?$AA?5?$AAs?$AAe?$AAt?$AA?5?$AAt?$AAo?$AA?5?$AAh?$AAi?$AAd?$AAe?$AA?5?$AAD?$AAa?$AAt?$AAa?$AA?5?$AAT?$AAa?$AAb@ 0010b4d0     sw_emext.obj
 0002:00001518       ??_C@_1EK@LEDAFMJA@?$AAR?$AAe?$AAg?$AAi?$AAs?$AAt?$AAr?$AAy?$AA?5?$AAi?$AAs?$AA?5?$AAs?$AAe?$AAt?$AA?5?$AAt?$AAo?$AA?5?$AAh?$AAi?$AAd?$AAe?$AA?5?$AAL?$AAo?$AAc?$AAa?$AAt?$AAi?$AAo?$AAn@ 0010b518     sw_emext.obj
 0002:00001564       ??_C@_1BO@CKHOGCJE@?$AA?4?$AA?2?$AAs?$AAw?$AA_?$AAe?$AAm?$AAe?$AAx?$AAt?$AA?4?$AAc?$AAp?$AAp?$AA?$AA@ 0010b564     sw_emext.obj
 0002:00001588       ??_C@_1GA@OPNDGMGH@?$AAC?$AAr?$AAe?$AAa?$AAt?$AAe?$AAE?$AAR?$AAI?$AAW?$AAi?$AAn?$AAd?$AAo?$AAw?$AA?5?$AA?5?$AAF?$AAa?$AAi?$AAl?$AAe?$AAd?$AA?5?$AAt?$AAo?$AA?5?$AAG?$AAe?$AAt?$AA?5?$AAP@ 0010b588     sw_emext.obj
 0002:000015e8       ??_C@_1CC@CKCHPABP@?$AAC?$AAS?$AAW?$AA_?$AAP?$AAh?$AAo?$AAn?$AAe?$AAE?$AAx?$AAt?$AAn?$AAE?$AAR?$AAI?$AA?$AA@ 0010b5e8     sw_emext.obj
 0002:00001610       ??_C@_1EI@HGHAGOCN@?$AAF?$AAa?$AAi?$AAl?$AA?5?$AAt?$AAo?$AA?5?$AAl?$AAa?$AAu?$AAn?$AAc?$AAh?$AA?5?$AAA?$AAA?$AAM?$AAG?$AA?4?$AAe?$AAx?$AAe?$AA?0?$AA?5?$AAe?$AAr?$AAr?$AAo?$AAr?$AA?5?$AA?$DN@ 0010b610     sw_emext.obj
 0002:00001658       ??_C@_1BC@NNIDFNKM@?$AAA?$AAA?$AAM?$AAG?$AA?4?$AAe?$AAx?$AAe?$AA?$AA@ 0010b658     sw_emext.obj
 0002:0000166c       ??_C@_15JNBOKNOG@?$AA?$AN?$AA?6?$AA?$AA@ 0010b66c     sw_emext.obj
 0002:00001674       ??_C@_1O@EFIFACDA@?$AA?$FL?$AAs?$AA?0?$AA?$CF?$AAs?$AA?$FN?$AA?$AA@ 0010b674     sw_emext.obj
 0002:00001684       ??_C@_1O@NCDIKDKD@?$AA?$FL?$AAb?$AA?0?$AA?$CF?$AAs?$AA?$FN?$AA?$AA@ 0010b684     sw_emext.obj
 0002:00001694       ??_C@_13JKNELIBG@?$AAT?$AA?$AA@ 0010b694     sw_emext.obj
 0002:00001698       ??_C@_13GAMECHAC@?$AAF?$AA?$AA@ 0010b698     sw_emext.obj
 0002:0000169c       ??_C@_1O@LNHJDFIO@?$AA?$FL?$AAi?$AA?0?$AA?$CF?$AAd?$AA?$FN?$AA?$AA@ 0010b69c     sw_emext.obj
 0002:000016ac       ??_C@_1BA@BEAEMJJN@?$AA?$FL?$AAu?$AAi?$AA?0?$AA?$CF?$AAd?$AA?$FN?$AA?$AA@ 0010b6ac     sw_emext.obj
 0002:000016bc       ??_C@_17FONKKNAB@?$AA?$FL?$AA?$DP?$AA?$FN?$AA?$AA@ 0010b6bc     sw_emext.obj
 0002:000016c8       ??_C@_1EE@JIPOFNAM@?$AAC?$AAS?$AAW?$AA_?$AAP?$AAh?$AAo?$AAn?$AAe?$AAE?$AAx?$AAt?$AAn?$AA?3?$AA?3?$AAI?$AAn?$AAv?$AAo?$AAk?$AAe?$AA?$CI?$AA?$CF?$AA2?$AA0?$AAs?$AA?5?$AA?$CI?$AA?$CF?$AA4?$AAd?$AA?$CJ@ 0010b6c8     sw_emext.obj
 0002:00001750       ??_C@_1CC@ICCBMOGN@?$AAP?$AAE?$AAD?$AAI?$AAS?$AAP?$AA_?$AAC?$AAA?$AAL?$AAL?$AAE?$AAR?$AA_?$AAI?$AAD?$AA?$AA@ 0010b750     sw_emext.obj
 0002:00001774       ??_C@_1CA@NAEGELEP@?$AAP?$AAE?$AAD?$AAI?$AAS?$AAP?$AA_?$AAI?$AAN?$AAC?$AAO?$AAM?$AAI?$AAN?$AAG?$AA?$AA@ 0010b774     sw_emext.obj
 0002:00001794       ??_C@_1BO@BNHBBGAA@?$AAP?$AAE?$AAD?$AAI?$AAS?$AAP?$AA_?$AAT?$AAA?$AAL?$AAK?$AAI?$AAN?$AAG?$AA?$AA@ 0010b794     sw_emext.obj
 0002:000017b4       ??_C@_1BI@LFFMLLEE@?$AAP?$AAE?$AAD?$AAI?$AAS?$AAP?$AA_?$AAH?$AAE?$AAL?$AAD?$AA?$AA@ 0010b7b4     sw_emext.obj
 0002:000017cc       ??_C@_1CC@BPAGALNB@?$AAP?$AAE?$AAD?$AAI?$AAS?$AAP?$AA_?$AAC?$AAO?$AAN?$AAN?$AAE?$AAC?$AAT?$AAE?$AAD?$AA?$AA@ 0010b7cc     sw_emext.obj
 0002:000017f0       ??_C@_1CK@NMCLONDB@?$AAP?$AAE?$AAD?$AAI?$AAS?$AAP?$AA_?$AAN?$AAE?$AAW?$AA_?$AAS?$AAI?$AAT?$AAE?$AA_?$AAH?$AAW?$AAN?$AAD?$AA?$AA@ 0010b7f0     sw_emext.obj
 0002:0000181c       ??_C@_1CA@IHKHEIPI@?$AAP?$AAE?$AAD?$AAI?$AAS?$AAP?$AA_?$AAC?$AAA?$AAL?$AAL?$AA_?$AAO?$AAI?$AAD?$AA?$AA@ 0010b81c     sw_emext.obj
 0002:00001840       ??_C@_1GO@OBOHBNMB@?$AAL?$AAo?$AAa?$AAd?$AAO?$AAe?$AAm?$AAD?$AAa?$AAt?$AAa?$AAI?$AAc?$AAo?$AAn?$AA?5?$AA?5?$AAG?$AAe?$AAt?$AAR?$AAi?$AAl?$AAS?$AAt?$AAa?$AAt?$AAu?$AAs?$AA?5?$AAf?$AAa@ 0010b840     sw_emext.obj
 0002:000018fc       ??_C@_1CC@HJFJDPII@?$AAS?$AAy?$AAs?$AAS?$AAe?$AAt?$AAt?$AAi?$AAn?$AAg?$AAs?$AAC?$AAl?$AAa?$AAs?$AAs?$AA?$AA@ 0010b8fc     syssettings.obj
 0002:00001920       ??_C@_1CE@HJEEKCON@?$AA?4?$AA?2?$AAs?$AAy?$AAs?$AAs?$AAe?$AAt?$AAt?$AAi?$AAn?$AAg?$AAs?$AA?4?$AAc?$AAp?$AAp?$AA?$AA@ 0010b920     syssettings.obj
 0002:00001944       ??_C@_1DE@HIADIKDF@?$AAI?$AAn?$AAi?$AAt?$AAS?$AAy?$AAs?$AAS?$AAe?$AAt?$AAt?$AAi?$AAn?$AAg?$AAs?$AAD?$AAl?$AAg?$AA?5?$AAF?$AAa?$AAi?$AAl?$AAe?$AAd?$AA?$AA@ 0010b944     syssettings.obj
 0002:00001978       ??_C@_1CI@NHCDLNLN@?$AAV?$AAe?$AAr?$AAs?$AAi?$AAo?$AAn?$AAI?$AAn?$AAf?$AAo?$AAD?$AAl?$AAg?$AAC?$AAl?$AAa?$AAs?$AAs?$AA?$AA@ 0010b978     versioninfo.obj
 0002:000019d8       ??_C@_1CK@DENEAOOB@?$AAM?$AAE?$AAI?$AAD?$AA?5?$AAi?$AAs?$AA?5?$AAn?$AAo?$AAt?$AA?5?$AAp?$AAr?$AAe?$AAs?$AAe?$AAn?$AAt?$AA?4?$AA?$AA@ 0010b9d8     versioninfo.obj
 0002:00001a04       ??_C@_17HDJIHIPC@?$AAN?$AA?1?$AAA?$AA?$AA@ 0010ba04     versioninfo.obj
 0002:00001a0c       ??_C@_15KNBIKKIN@?$AA?$CF?$AAd?$AA?$AA@ 0010ba0c     versioninfo.obj
 0002:00001a14       ??_C@_15GANGMFKL@?$AA?$CF?$AAs?$AA?$AA@ 0010ba14     versioninfo.obj
 0002:00001a20       ??_C@_1HM@DBKPLNBD@?$AAD?$AAo?$AA?5?$AAn?$AAo?$AAt?$AA?5?$AAl?$AAo?$AAa?$AAd?$AA?5?$AAa?$AAn?$AAy?$AAt?$AAh?$AAi?$AAn?$AAg?$AA?4?$AA?4?$AA?4?$AA?4?$AAt?$AAh?$AAi?$AAs?$AA?5?$AAv?$AAe?$AAr@ 0010ba20     versioninfo.obj
 0002:00001aa0       ??_C@_1HK@CBBKEHKD@?$AAD?$AAo?$AA?5?$AAn?$AAo?$AAt?$AA?5?$AAl?$AAo?$AAa?$AAd?$AA?5?$AAa?$AAn?$AAy?$AAt?$AAh?$AAi?$AAn?$AAg?$AA?4?$AA?4?$AA?4?$AA?4?$AAt?$AAh?$AAi?$AAs?$AA?5?$AAv?$AAe?$AAr@ 0010baa0     versioninfo.obj
 0002:00001b1c       ??_C@_1CE@PALBMHKD@?$AA?4?$AA?2?$AAv?$AAe?$AAr?$AAs?$AAi?$AAo?$AAn?$AAi?$AAn?$AAf?$AAo?$AA?4?$AAc?$AAp?$AAp?$AA?$AA@ 0010bb1c     versioninfo.obj
 0002:00001b40       ??_C@_1LA@NDBKELK@?$AAD?$AAo?$AA?5?$AAn?$AAo?$AAt?$AA?5?$AAl?$AAo?$AAa?$AAd?$AA?5?$AAa?$AAn?$AAy?$AAt?$AAh?$AAi?$AAn?$AAg?$AA?4?$AA?4?$AA?4?$AA?4?$AAt?$AAh?$AAi?$AAs?$AA?5?$AAv?$AAe?$AAr@ 0010bb40     versioninfo.obj
 0002:00001bf0       ??_C@_1DE@ONINLNPH@?$AAI?$AAn?$AAi?$AAt?$AAV?$AAe?$AAr?$AAs?$AAi?$AAo?$AAn?$AAI?$AAn?$AAf?$AAo?$AAD?$AAl?$AAg?$AA?5?$AAF?$AAa?$AAi?$AAl?$AAe?$AAd?$AA?$AA@ 0010bbf0     versioninfo.obj
 0002:00001c24       IID_IShellPropSheetExt     0010bc24     uuid:shguids_guid29.obj
 0002:00001c34       IID_IDispatch              0010bc34     uuid:oaidl_i_guid4.obj
 0002:00001c44       IID_IShellExtInit          0010bc44     uuid:shguids_guid28.obj
 0002:00001d20       __IMPORT_DESCRIPTOR_commctrl 0010bd20     commctrl:commctrl.dll
 0002:00001d34       __IMPORT_DESCRIPTOR_COREDLL 0010bd34     coredll:COREDLL.dll
 0002:00001d48       __IMPORT_DESCRIPTOR_sw_utilityG 0010bd48     sw_utilityG:sw_utilityG.dll
 0002:00001d5c       __IMPORT_DESCRIPTOR_GobiApi 0010bd5c     gobiapi:GobiApi.dll
 0002:00001d70       __IMPORT_DESCRIPTOR_cellcore 0010bd70     cellcore:cellcore.dll
 0002:00001d84       __NULL_IMPORT_DESCRIPTOR   0010bd84     commctrl:commctrl.dll
 0003:00000000       __imp_UpdateWindow         0010d000     coredll:COREDLL.dll
 0003:00000004       __imp_EnableWindow         0010d004     coredll:COREDLL.dll
 0003:00000008       __imp_GetDlgItem           0010d008     coredll:COREDLL.dll
 0003:0000000c       __imp_ShowWindow           0010d00c     coredll:COREDLL.dll
 0003:00000010       __imp_SetWindowTextW       0010d010     coredll:COREDLL.dll
 0003:00000014       __imp_LoadStringW          0010d014     coredll:COREDLL.dll
 0003:00000018       __imp_wcscat               0010d018     coredll:COREDLL.dll
 0003:0000001c       __imp_MessageBoxW          0010d01c     coredll:COREDLL.dll
 0003:00000020       __imp_GetLastError         0010d020     coredll:COREDLL.dll
 0003:00000024       __imp_CreateProcessW       0010d024     coredll:COREDLL.dll
 0003:00000028       __imp_SetFocus             0010d028     coredll:COREDLL.dll
 0003:0000002c       __imp_EndDialog            0010d02c     coredll:COREDLL.dll
 0003:00000030       __imp_swprintf             0010d030     coredll:COREDLL.dll
 0003:00000034       __imp_RegisterClassW       0010d034     coredll:COREDLL.dll
 0003:00000038       __imp_GetStockObject       0010d038     coredll:COREDLL.dll
 0003:0000003c       __imp_memset               0010d03c     coredll:COREDLL.dll
 0003:00000040       __imp_RegisterWindowMessageW 0010d040     coredll:COREDLL.dll
 0003:00000044       __imp_SetWindowPos         0010d044     coredll:COREDLL.dll
 0003:00000048       __imp_GetClientRect        0010d048     coredll:COREDLL.dll
 0003:0000004c       __imp_SendMessageW         0010d04c     coredll:COREDLL.dll
 0003:00000050       __imp_SendDlgItemMessageW  0010d050     coredll:COREDLL.dll
 0003:00000054       __imp_RegCloseKey          0010d054     coredll:COREDLL.dll
 0003:00000058       __imp_RegQueryValueExW     0010d058     coredll:COREDLL.dll
 0003:0000005c       __imp_RegOpenKeyExW        0010d05c     coredll:COREDLL.dll
 0003:00000060       __imp_RegSetValueExW       0010d060     coredll:COREDLL.dll
 0003:00000064       __imp_RegCreateKeyExW      0010d064     coredll:COREDLL.dll
 0003:00000068       __imp_NKDbgPrintfW         0010d068     coredll:COREDLL.dll
 0003:0000006c       __imp_wsprintfW            0010d06c     coredll:COREDLL.dll
 0003:00000070       __imp__isctype             0010d070     coredll:COREDLL.dll
 0003:00000074       __imp_wcslen               0010d074     coredll:COREDLL.dll
 0003:00000078       __imp_KillTimer            0010d078     coredll:COREDLL.dll
 0003:0000007c       __imp_LocalAlloc           0010d07c     coredll:COREDLL.dll
 0003:00000080       __imp_GetWindowTextW       0010d080     coredll:COREDLL.dll
 0003:00000084       __imp_malloc               0010d084     coredll:COREDLL.dll
 0003:00000088       __imp_WideCharToMultiByte  0010d088     coredll:COREDLL.dll
 0003:0000008c       __imp_free                 0010d08c     coredll:COREDLL.dll
 0003:00000090       __imp_strcpy               0010d090     coredll:COREDLL.dll
 0003:00000094       __imp_memcpy               0010d094     coredll:COREDLL.dll
 0003:00000098       __imp_LoadLibraryW         0010d098     coredll:COREDLL.dll
 0003:0000009c       __imp_GetWindowRect        0010d09c     coredll:COREDLL.dll
 0003:000000a0       __imp_SetWindowLongW       0010d0a0     coredll:COREDLL.dll
 0003:000000a4       __imp_GetWindowLongW       0010d0a4     coredll:COREDLL.dll
 0003:000000a8       __imp_memcmp               0010d0a8     coredll:COREDLL.dll
 0003:000000ac       __imp_GetModuleFileNameW   0010d0ac     coredll:COREDLL.dll
 0003:000000b0       __imp_GetModuleHandleW     0010d0b0     coredll:COREDLL.dll
 0003:000000b4       __imp_RegDeleteKeyW        0010d0b4     coredll:COREDLL.dll
 0003:000000b8       __imp__purecall            0010d0b8     coredll:COREDLL.dll
 0003:000000bc       __imp_PostMessageW         0010d0bc     coredll:COREDLL.dll
 0003:000000c0       __imp_RemoveProp           0010d0c0     coredll:COREDLL.dll
 0003:000000c4       __imp_GetActiveWindow      0010d0c4     coredll:COREDLL.dll
 0003:000000c8       __imp_wcscpy               0010d0c8     coredll:COREDLL.dll
 0003:000000cc       __imp_EndPaint             0010d0cc     coredll:COREDLL.dll
 0003:000000d0       __imp_DrawTextW            0010d0d0     coredll:COREDLL.dll
 0003:000000d4       __imp_ExtTextOutW          0010d0d4     coredll:COREDLL.dll
 0003:000000d8       __imp_BeginPaint           0010d0d8     coredll:COREDLL.dll
 0003:000000dc       __imp_DefWindowProcW       0010d0dc     coredll:COREDLL.dll
 0003:000000e0       __imp_InvalidateRect       0010d0e0     coredll:COREDLL.dll
 0003:000000e4       __imp_CreateWindowExW      0010d0e4     coredll:COREDLL.dll
 0003:000000e8       __imp_InterlockedCompareExchange 0010d0e8     coredll:COREDLL.dll
 0003:000000ec       __imp_LoadIconW            0010d0ec     coredll:COREDLL.dll
 0003:000000f0       __imp_DestroyIcon          0010d0f0     coredll:COREDLL.dll
 0003:000000f4       __imp_??3@YAXPAX@Z         0010d0f4     coredll:COREDLL.dll
 0003:000000f8       __imp_??2@YAPAXI@Z         0010d0f8     coredll:COREDLL.dll
 0003:000000fc       __imp_wcsncpy              0010d0fc     coredll:COREDLL.dll
 0003:00000100       __imp_TlsGetValue          0010d100     coredll:COREDLL.dll
 0003:00000104       __imp_SetTimer             0010d104     coredll:COREDLL.dll
 0003:00000108       __imp_CreateThread         0010d108     coredll:COREDLL.dll
 0003:0000010c       __imp_TlsSetValue          0010d10c     coredll:COREDLL.dll
 0003:00000110       __imp_TlsCall              0010d110     coredll:COREDLL.dll
 0003:00000114       __imp_memmove              0010d114     coredll:COREDLL.dll
 0003:00000118       __imp___C_specific_handler 0010d118     coredll:COREDLL.dll
 0003:0000011c       __imp_?terminate@std@@YAXXZ 0010d11c     coredll:COREDLL.dll
 0003:00000120       __imp_strcmp               0010d120     coredll:COREDLL.dll
 0003:00000124       __imp___security_gen_cookie 0010d124     coredll:COREDLL.dll
 0003:00000128       __imp_LocalFree            0010d128     coredll:COREDLL.dll
 0003:0000012c       __imp___report_gsfailure   0010d12c     coredll:COREDLL.dll
 0003:00000130       \177COREDLL_NULL_THUNK_DATA 0010d130     coredll:COREDLL.dll
 0003:00000134       __imp_UIMVerifyPIN         0010d134     gobiapi:GobiApi.dll
 0003:00000138       __imp_UIMGetCardStatus     0010d138     gobiapi:GobiApi.dll
 0003:0000013c       __imp_UIMSetPINProtection  0010d13c     gobiapi:GobiApi.dll
 0003:00000140       __imp_UIMUnblockPIN        0010d140     gobiapi:GobiApi.dll
 0003:00000144       __imp_UIMChangePIN         0010d144     gobiapi:GobiApi.dll
 0003:00000148       __imp_QCWWANDisconnect     0010d148     gobiapi:GobiApi.dll
 0003:0000014c       __imp_QCWWANConnect        0010d14c     gobiapi:GobiApi.dll
 0003:00000150       __imp_SwiSetDeviceRemovalCallback 0010d150     gobiapi:GobiApi.dll
 0003:00000154       __imp_GetCDMANetworkParameters 0010d154     gobiapi:GobiApi.dll
 0003:00000158       __imp_SetCDMANetworkParameters 0010d158     gobiapi:GobiApi.dll
 0003:0000015c       __imp_GetRTREConfig        0010d15c     gobiapi:GobiApi.dll
 0003:00000160       \177GobiApi_NULL_THUNK_DATA 0010d160     gobiapi:GobiApi.dll
 0003:00000164       __imp_tapiRequestMakeCallW 0010d164     cellcore:cellcore.dll
 0003:00000168       \177cellcore_NULL_THUNK_DATA 0010d168     cellcore:cellcore.dll
 0003:0000016c       __imp_CreatePropertySheetPageW 0010d16c     commctrl:commctrl.dll
 0003:00000170       __imp_DestroyPropertySheetPage 0010d170     commctrl:commctrl.dll
 0003:00000174       \177commctrl_NULL_THUNK_DATA 0010d174     commctrl:commctrl.dll
 0003:00000178       __imp_?GetAutoUpdateTimeUI@@YAKXZ 0010d178     sw_utilityG:sw_utilityG.dll
 0003:0000017c       __imp_?SetCallGuardReg@@YAXK@Z 0010d17c     sw_utilityG:sw_utilityG.dll
 0003:00000180       __imp_GetVersionInfo       0010d180     sw_utilityG:sw_utilityG.dll
 0003:00000184       __imp_?GetAutoUpdateTime@@YAKXZ 0010d184     sw_utilityG:sw_utilityG.dll
 0003:00000188       __imp_?SetAutoUpdateTime@@YAXH@Z 0010d188     sw_utilityG:sw_utilityG.dll
 0003:0000018c       __imp_?GetCallGuardReg@@YAKXZ 0010d18c     sw_utilityG:sw_utilityG.dll
 0003:00000190       __imp_?GetCarrierIndex@@YAKXZ 0010d190     sw_utilityG:sw_utilityG.dll
 0003:00000194       __imp_?LogV@@YAXPBGZZ      0010d194     sw_utilityG:sw_utilityG.dll
 0003:00000198       __imp_?GetVerInfo@@YAPAGPAUHINSTANCE__@@@Z 0010d198     sw_utilityG:sw_utilityG.dll
 0003:0000019c       __imp_?InitLog@@YAXPAUHINSTANCE__@@@Z 0010d19c     sw_utilityG:sw_utilityG.dll
 0003:000001a0       __imp_ModGetPreferredPrivacyMode 0010d1a0     sw_utilityG:sw_utilityG.dll
 0003:000001a4       __imp_ModGetRoamStatus     0010d1a4     sw_utilityG:sw_utilityG.dll
 0003:000001a8       __imp_ModGetLocationStatus 0010d1a8     sw_utilityG:sw_utilityG.dll
 0003:000001ac       __imp_ModGetRoamingMode    0010d1ac     sw_utilityG:sw_utilityG.dll
 0003:000001b0       __imp_ModSetRoamingMode    0010d1b0     sw_utilityG:sw_utilityG.dll
 0003:000001b4       __imp_ModSetPreferredPrivacyMode 0010d1b4     sw_utilityG:sw_utilityG.dll
 0003:000001b8       __imp_ModSetLocationMode   0010d1b8     sw_utilityG:sw_utilityG.dll
 0003:000001bc       __imp_?SetWaitCursor@@YAXXZ 0010d1bc     sw_utilityG:sw_utilityG.dll
 0003:000001c0       __imp_?SetNormalCursor@@YAXXZ 0010d1c0     sw_utilityG:sw_utilityG.dll
 0003:000001c4       __imp_GetOMADMConfig       0010d1c4     sw_utilityG:sw_utilityG.dll
 0003:000001c8       __imp_?InWideMode@@YAHXZ   0010d1c8     sw_utilityG:sw_utilityG.dll
 0003:000001cc       __imp_?RelayoutDialog@@YAHPAUHINSTANCE__@@PAUHWND__@@PBG@Z 0010d1cc     sw_utilityG:sw_utilityG.dll
 0003:000001d0       __imp_?LogC@@YAXPBGZZ      0010d1d0     sw_utilityG:sw_utilityG.dll
 0003:000001d4       __imp_?LogStoreFileLine@@YAXPAGH@Z 0010d1d4     sw_utilityG:sw_utilityG.dll
 0003:000001d8       __imp_?SetConnectionProfile@@YAJXZ 0010d1d8     sw_utilityG:sw_utilityG.dll
 0003:000001dc       __imp_GetLogoTestReg       0010d1dc     sw_utilityG:sw_utilityG.dll
 0003:000001e0       __imp_GetRilStatus         0010d1e0     sw_utilityG:sw_utilityG.dll
 0003:000001e4       __imp_?GetProductFeatures@@YAHAAK@Z 0010d1e4     sw_utilityG:sw_utilityG.dll
 0003:000001e8       __imp_SetEquipmentState    0010d1e8     sw_utilityG:sw_utilityG.dll
 0003:000001ec       \177sw_utilityG_NULL_THUNK_DATA 0010d1ec     sw_utilityG:sw_utilityG.dll
 0003:000001f0       __xc_a                     0010d1f0     corelibc:crt0init.obj
 0003:0000023c       __xc_z                     0010d23c     corelibc:crt0init.obj
 0003:00000240       __xi_a                     0010d240     corelibc:crt0init.obj
 0003:00000244       __xi_z                     0010d244     corelibc:crt0init.obj
 0003:00000248       __xp_a                     0010d248     corelibc:crt0init.obj
 0003:0000024c       __xp_z                     0010d24c     corelibc:crt0init.obj
 0003:00000250       __xt_a                     0010d250     corelibc:crt0init.obj
 0003:00000254       __xt_z                     0010d254     corelibc:crt0init.obj
 0003:00000258       ?g_szDataClass@@3PAGA      0010d258     data.obj
 0003:0000025c       ?g_szDatalistClass@@3PAGA  0010d25c     datalist.obj
 0003:00000260       ?g_szLocationClass@@3PAGA  0010d260     location.obj
 0003:00000264       ?g_szPhsListClass@@3PAGA   0010d264     phs_list.obj
 0003:0000026c       ?g_sz_RUIM_CALL_CTRL_DlgClass@@3PAGA 0010d26c     ruim_call_ctrl.obj
 0003:00000274       ?g_sz_RUIM_PIN_DlgClass@@3PAGA 0010d274     ruim_pin.obj
 0003:00000278       ?PinStateText@@3PAPAGA     0010d278     ruim_pin.obj
 0003:00000294       ?g_sz_SPRINT_ROAMING_OPTION_DlgClass@@3PAGA 0010d294     Sprint_roaming_option.obj
 0003:00000298       ?MY_NOTIFYICON@@3IA        0010d298     sw_emext.obj
 0003:0000029c       ?g_szSysSettingsClass@@3PAGA 0010d29c     syssettings.obj
 0003:000002a4       ?g_szVersionInfoDlgClass@@3PAGA 0010d2a4     versioninfo.obj
 0003:000002a8       __security_cookie_complement 0010d2a8     corelibc:seccook.obj
 0003:000002ac       __security_cookie          0010d2ac     corelibc:seccook.obj
 0003:000002bc       ?g_hWndDataList@@3PAUHWND__@@A 0010d2bc     datalist.obj
 0003:000002c0       ?g_bProvision@@3HA         0010d2c0     datalist.obj
 0003:000002c4       ?g_bReset@@3HA             0010d2c4     datalist.obj
 0003:000002cc       ?g_hWndPhsList@@3PAUHWND__@@A 0010d2cc     phs_list.obj
 0003:000002d0       ?g_hWndMainList@@3PAUHWND__@@A 0010d2d0     phs_list.obj
 0003:000002d8       ?g_CallCrlTimer@@3IA       0010d2d8     ruim_call_ctrl.obj
 0003:000002e8       ?gPIN1State@@3EA           0010d2e8     ruim_pin.obj
 0003:000002ec       ?gDialog@@3PAUHWND__@@A    0010d2ec     ruim_pin.obj
 0003:00000318       ?g_szBuffer@@3PAGA         0010d318     sw_emext.obj
 0003:000012b8       ?g_hCurrentWnd@@3PAUHWND__@@A 0010e2b8     sw_emext.obj
 0003:000012bc       ?g_nCarrier@@3KA           0010e2bc     sw_emext.obj
 0003:000012c0       ?g_Err@@3UtagErrorInfo@@A  0010e2c0     sw_emext.obj
 0003:000014c8       ?g_stRilStatus@@3USW_RILStatus@@A 0010e4c8     sw_emext.obj
 0003:00001508       ?g_hResInst@@3PAUHINSTANCE__@@A 0010e508     sw_emext.obj
 0003:0000150c       ?g_hInst@@3PAUHINSTANCE__@@A 0010e50c     sw_emext.obj
 0003:00001510       ?g_dwDLLRefCount@@3IA      0010e510     sw_emext.obj
 0003:00001514       ?g_hwndERI@@3PAUHWND__@@A  0010e514     sw_emext.obj
 0003:00001518       ?g_dwLen@@3KA              0010e518     sw_emext.obj
 0003:0000151c       ?gGobiConnected@@3HA       0010e51c     sw_emext.obj
 0003:00001520       ?g_RUIMRefreshTimer@@3IA   0010e520     sw_emext.obj
 0003:00001524       ?g_RoamRefreshTimer@@3IA   0010e524     sw_emext.obj
 0003:00001528       ?g_DeviceSearchTimer@@3IA  0010e528     sw_emext.obj
 0003:0000152c       ?g_hIconDormant@@3PAUHICON__@@A 0010e52c     sw_emext.obj
 0003:00001530       ?g_hIconRevA@@3PAUHICON__@@A 0010e530     sw_emext.obj
 0003:00001534       ?g_hDlg@@3PAUHWND__@@A     0010e534     sw_emext.obj
 0003:00001548       ?g_VersionInfo@@3UtagRILVERNOINFO@@A 0010e548     versioninfo.obj
 0003:00002158       __onexitend                0010f158     <common>
 0003:0000215c       __onexitbegin              0010f15c     <common>
 0003:00002160       _exitflag                  0010f160     <common>
 0003:00002164       _pRawDllMain               0010f164     <common>

 entry point at        0001:00007158

 Static symbols

 0001:00002af4       ?WriteDWORDValue@@YAJPAUHKEY__@@PBG1K@Z 00103af4 f   Sprint_roaming_option.obj
 0001:000037fc       ?DeviceRemovalCallback@@YAXK@Z 001047fc f   sw_emext.obj
 0001:00004ecc       __unwind$43329             00105ecc f   sw_emext.obj
 0001:000072b4       doexit                     001082b4 f   corelibc:crt0dat.obj
 0001:0000768c       ?CanThisExceptionObjectBeDestructed@@YAEPAUEHExceptionRecord@@E@Z 0010868c f   LIBCMT:frame_ce.obj
 0001:000079d8       ?CallCatchBlock@@YAPAXPAUEHExceptionRecord@@PAKPAU_CONTEXT@@PBU_s_FuncInfo@@PAXHK@Z 001089d8 f   LIBCMT:frame_ce.obj
 0001:00007d70       ?BuildCatchObject@@YAXPAUEHExceptionRecord@@PAKPBU_s_HandlerType@@PBU_s_CatchableType@@@Z 00108d70 f   LIBCMT:frame_ce.obj
 0001:00007f44       ?FindHandler@@YAEPAUEHExceptionRecord@@PAKPAU_CONTEXT@@PAU_DISPATCHER_CONTEXT@@PBU_s_FuncInfo@@H@Z 00108f44 f   LIBCMT:frame_ce.obj
 0001:000087e8       ??__ERIL_STATUS_CHANGED@@YAXXZ 001097e8 f   data.obj
 0001:00008808       ??__ERIL_STATUS_CHANGED@@YAXXZ 00109808 f   location.obj
 0001:00008828       ??__ERIL_STATUS_CHANGED@@YAXXZ 00109828 f   ruim_call_ctrl.obj
 0001:00008848       ??__ERIL_DBG_NOTIFY@@YAXXZ 00109848 f   ruim_call_ctrl.obj
 0001:00008868       ??__ERIL_SET_ERITEXT@@YAXXZ 00109868 f   ruim_call_ctrl.obj
 0001:00008888       ??__ERIL_STATUS_CHANGED@@YAXXZ 00109888 f   ruim_pin.obj
 0001:000088a8       ??__ERIL_DBG_NOTIFY@@YAXXZ 001098a8 f   ruim_pin.obj
 0001:000088c8       ??__ERIL_SET_ERITEXT@@YAXXZ 001098c8 f   ruim_pin.obj
 0001:000088e8       ??__ERIL_STATUS_CHANGED@@YAXXZ 001098e8 f   Sprint_roaming_option.obj
 0001:00008908       ??__ERIL_DBG_NOTIFY@@YAXXZ 00109908 f   Sprint_roaming_option.obj
 0001:00008928       ??__ERIL_SET_ERITEXT@@YAXXZ 00109928 f   Sprint_roaming_option.obj
 0001:00008948       ??__ERIL_STATUS_CHANGED@@YAXXZ 00109948 f   stdafx.obj
 0001:00008968       ??__ERIL_DBG_NOTIFY@@YAXXZ 00109968 f   stdafx.obj
 0001:00008988       ??__ERIL_SET_ERITEXT@@YAXXZ 00109988 f   stdafx.obj
 0001:000089a8       ??__ERIL_STATUS_CHANGED@@YAXXZ 001099a8 f   sw_emext.obj
 0001:000089c8       ??__ERIL_SET_ERITEXT@@YAXXZ 001099c8 f   sw_emext.obj
 0001:000089e8       ??__ERIL_STATUS_CHANGED@@YAXXZ 001099e8 f   syssettings.obj
